:020000040000FA
:10000000003065000515392090309D0018203C30E7
:100010009D0018207F309D001820392080309D00E1
:1000200018203C309D0018207F309D0018200328A8
:10003000051118309F009F0B1B2808309B009D0C5A
:1000400003182528000005112828051500000000C8
:1000500017309F009F0B2A289B0B1F2800000000D1
:1000600000000000000005151A309F009F0B362885
:1000700008000D309C00FF309B00FF309A009A0B67
:0C0080003F289B0B3D289C0B3B280800F0
:02400E00F23F7F
:00000001FF
